:020000040000FA
:02000000602876
:08000800C000030EC1008B1CB7
:1000100029288B10261B1B2885162208071AA000EA
:100020001030071AA100A10B2F281030A100A00B3F
:100030002F282614292885122208071EA000103018
:10004000071EA100A10B2F281030A100A00B2F2804
:1000500026140B1D2F280B110508203A8500410E90
:080060008300C00E400E0900F0
:1000C000A0011030A100A201A601C001C101831648
:1000D000051085100515851505128516071487145A
:1000E00007158715071687128312850187010730C8
:1000F0009900873083168100831200309000003011
:1001000083168C008312F0308B00831685128312C5
:100110008512831685168312851A2617851E2613C7
:1001200083168512831264009E20261C9328051DC9
:100130009328261087160000871293280039071C81
:100140000838871C0438071D0238871D0138013E16
:04015000A200080001
:084000000000000001000200B5
:02400E00CC01E3
:00000001FF
